 localtab005

 Timestamp is 79ede828 (reproducible build file hash)

 Preferred load address is 0000000180000000

 Start         Length     Name                   Class
 0001:00000000 000035e0H .text$mn                CODE
 0001:000035e0 00000036H .text$mn$00             CODE
 0001:00003616 00000092H .text$x                 CODE
 0002:00000000 000001c8H .idata$5                DATA
 0002:000001c8 00000038H .00cfg                  DATA
 0002:00000200 00000008H .CRT$XCA                DATA
 0002:00000208 00000008H .CRT$XCZ                DATA
 0002:00000210 00000008H .CRT$XIA                DATA
 0002:00000218 00000008H .CRT$XIC                DATA
 0002:00000220 00000008H .CRT$XIZ                DATA
 0002:00000228 00000008H .CRT$XLA                DATA
 0002:00000230 00000008H .CRT$XLZ                DATA
 0002:00000238 00000008H .CRT$XPA                DATA
 0002:00000240 00000008H .CRT$XPZ                DATA
 0002:00000248 00000008H .CRT$XTA                DATA
 0002:00000250 00000010H .CRT$XTZ                DATA
 0002:00000258 00000000H .gehcont$y              DATA
 0002:00000258 00000000H .gfids$y                DATA
 0002:00000260 000025a0H .rdata                  DATA
 0002:00002800 00000000H .rdata$CastGuardVftablesA DATA
 0002:00002800 00000000H .rdata$CastGuardVftablesC DATA
 0002:00002800 00000028H .rdata$T                DATA
 0002:00002828 000000a8H .rdata$voltmd           DATA
 0002:000028d0 00000318H .rdata$zzzdbg           DATA
 0002:00002be8 00000008H .rtc$IAA                DATA
 0002:00002bf0 00000008H .rtc$IZZ                DATA
 0002:00002bf8 00000008H .rtc$TAA                DATA
 0002:00002c00 00000008H .rtc$TZZ                DATA
 0002:00002c08 00000004H .tls                    DATA
 0002:00002c0c 00000004H .tls$                   DATA
 0002:00002c10 00000008H .tls$ZZZ                DATA
 0002:00002c18 00000318H .xdata                  DATA
 0002:00002f30 000003a4H .edata                  DATA
 0002:000032d4 0000008cH .idata$2                DATA
 0002:00003360 00000018H .idata$3                DATA
 0002:00003378 000001c8H .idata$4                DATA
 0002:00003540 00000486H .idata$6                DATA
 0003:00000000 000002f0H .data                   DATA
 0003:000002f0 0001b248H .bss                    DATA
 0004:00000000 000003b4H .pdata                  DATA

  Address         Publics by Value              Rva+Base               Lib:Object

 0000:00000000       __AbsoluteZero             0000000000000000     <absolute>
 0000:00000000       ___safe_se_handler_count   0000000000000000     <absolute>
 0000:00000000       ___safe_se_handler_table   0000000000000000     <absolute>
 0000:00000000       __arm64x_extra_rfe_table   0000000000000000     <absolute>
 0000:00000000       __arm64x_extra_rfe_table_size 0000000000000000     <absolute>
 0000:00000000       __arm64x_native_entrypoint 0000000000000000     <absolute>
 0000:00000000       __arm64x_redirection_metadata 0000000000000000     <absolute>
 0000:00000000       __arm64x_redirection_metadata_count 0000000000000000     <absolute>
 0000:00000000       __dynamic_value_reloc_table 0000000000000000     <absolute>
 0000:00000000       __enclave_config           0000000000000000     <absolute>
 0000:00000000       __guard_check_icall_a64n_fptr 0000000000000000     <absolute>
 0000:00000000       __guard_eh_cont_count      0000000000000000     <absolute>
 0000:00000000       __guard_eh_cont_table      0000000000000000     <absolute>
 0000:00000000       __guard_fids_count         0000000000000000     <absolute>
 0000:00000000       __guard_fids_table         0000000000000000     <absolute>
 0000:00000000       __guard_iat_count          0000000000000000     <absolute>
 0000:00000000       __guard_iat_table          0000000000000000     <absolute>
 0000:00000000       __guard_longjmp_count      0000000000000000     <absolute>
 0000:00000000       __guard_longjmp_table      0000000000000000     <absolute>
 0000:00000000       __hybrid_auxiliary_iat     0000000000000000     <absolute>
 0000:00000000       __hybrid_auxiliary_iat_copy 0000000000000000     <absolute>
 0000:00000000       __hybrid_code_map          0000000000000000     <absolute>
 0000:00000000       __hybrid_code_map_count    0000000000000000     <absolute>
 0000:00000000       __x64_code_ranges_to_entry_points 0000000000000000     <absolute>
 0000:00000000       __x64_code_ranges_to_entry_points_count 0000000000000000     <absolute>
 0000:00000100       __guard_flags              0000000000000100     <absolute>
 0000:00000000       __ImageBase                0000000180000000     <linker-defined>
 0001:00000000       ?NewObject@JNIEnv_@@QEAAPEAV_jobject@@PEAV_jclass@@PEAU_jmethodID@@ZZ 0000000180001000 f i liblocaltab005.obj
 0001:00000028       ?TranslateError@@YAPEBDW4jvmtiError@@@Z 0000000180001028 f   liblocaltab005.obj
 0001:000002e0       ?nsk_jni_check_exception@@YAHPEAUJNIEnv_@@QEBDH@Z 00000001800012e0 f   liblocaltab005.obj
 0001:00000424       ?nsk_jni_lverify@@YAHHPEAUJNIEnv_@@HQEBDH1ZZ 0000000180001424 f   liblocaltab005.obj
 0001:000004c4       Agent_Initialize           00000001800014c4 f   liblocaltab005.obj
 0001:000006b4       Agent_OnAttach             00000001800016b4 f   liblocaltab005.obj
 0001:000006b4       Agent_OnLoad               00000001800016b4 f   liblocaltab005.obj
 0001:000006bc       Java_nsk_jvmti_GetLocalVariableTable_localtab005_check 00000001800016bc f   liblocaltab005.obj
 0001:000006fc       Java_nsk_jvmti_unit_FollowReferences_FollowRefObjects_addRefToVerify 00000001800016fc f   liblocaltab005.obj
 0001:000008d4       Java_nsk_jvmti_unit_FollowReferences_FollowRefObjects_getTag 00000001800018d4 f   liblocaltab005.obj
 0001:00000994       Java_nsk_jvmti_unit_FollowReferences_FollowRefObjects_resetRefsToVerify 0000000180001994 f   liblocaltab005.obj
 0001:0000099c       Java_nsk_jvmti_unit_FollowReferences_FollowRefObjects_resetTags 000000018000199c f   liblocaltab005.obj
 0001:000009e0       Java_nsk_jvmti_unit_FollowReferences_FollowRefObjects_setTag 00000001800019e0 f   liblocaltab005.obj
 0001:00000c38       Java_nsk_share_jvmti_ArgumentHandler_getAgentOptionsString 0000000180001c38 f   liblocaltab005.obj
 0001:00000ce8       Java_nsk_share_jvmti_DebugeeClass_checkStatus 0000000180001ce8 f   liblocaltab005.obj
 0001:00000d70       Java_nsk_share_jvmti_DebugeeClass_resetAgentData 0000000180001d70 f   liblocaltab005.obj
 0001:00000dd0       Java_nsk_share_jvmti_RedefineAgent_agentStatus 0000000180001dd0 f   liblocaltab005.obj
 0001:00000ddc       Java_nsk_share_jvmti_RedefineAgent_isRedefined 0000000180001ddc f   liblocaltab005.obj
 0001:00000de8       Java_nsk_share_jvmti_RedefineAgent_redefineAttempted 0000000180001de8 f   liblocaltab005.obj
 0001:00000df4       MA_checkStatus             0000000180001df4 f   liblocaltab005.obj
 0001:00000e98       __local_stdio_printf_options 0000000180001e98 f i liblocaltab005.obj
 0001:0000174c       exitOnError                000000018000274c f   liblocaltab005.obj
 0001:00001800       fprintf                    0000000180002800 f i liblocaltab005.obj
 0001:00001844       nsk_complain               0000000180002844 f   liblocaltab005.obj
 0001:00001870       nsk_jvmti_createJVMTIEnv   0000000180002870 f   liblocaltab005.obj
 0001:000019a0       nsk_jvmti_lverify          00000001800029a0 f   liblocaltab005.obj
 0001:00001a90       nsk_jvmti_parseOptions     0000000180002a90 f   liblocaltab005.obj
 0001:00001ce0       nsk_jvmti_resetAgentData   0000000180002ce0 f   liblocaltab005.obj
 0001:00001d60       nsk_jvmti_setFailStatus    0000000180002d60 f   liblocaltab005.obj
 0001:00001d9c       nsk_lcomplain              0000000180002d9c f   liblocaltab005.obj
 0001:00001dbc       nsk_ldisplay               0000000180002dbc f   liblocaltab005.obj
 0001:00001ddc       nsk_ltrace                 0000000180002ddc f   liblocaltab005.obj
 0001:00001dfc       nsk_lvcomplain             0000000180002dfc f   liblocaltab005.obj
 0001:00001fb4       nsk_lvdisplay              0000000180002fb4 f   liblocaltab005.obj
 0001:00002000       nsk_lverify                0000000180003000 f   liblocaltab005.obj
 0001:0000205c       nsk_lvtrace                000000018000305c f   liblocaltab005.obj
 0001:000020bc       nsk_printf                 00000001800030bc f   liblocaltab005.obj
 0001:000020e4       nsk_vprintf                00000001800030e4 f   liblocaltab005.obj
 0001:00002198       printf                     0000000180003198 f i liblocaltab005.obj
 0001:000026c0       __raise_securityfailure    00000001800036c0 f   MSVCRT:gs_report.obj
 0001:000026f4       __report_gsfailure         00000001800036f4 f   MSVCRT:gs_report.obj
 0001:00002934       __GSHandlerCheck           0000000180003934 f   MSVCRT:gshandler.obj
 0001:00002954       __GSHandlerCheckCommon     0000000180003954 f   MSVCRT:gshandler.obj
 0001:000029c0       __security_check_cookie    00000001800039c0 f   MSVCRT:amdsecgs.obj
 0001:00002d00       _DllMainCRTStartup         0000000180003d00 f   MSVCRT:dll_dllmain.obj
 0001:00002d40       __scrt_acquire_startup_lock 0000000180003d40 f   MSVCRT:utility.obj
 0001:00002d7c       __scrt_dllmain_after_initialize_c 0000000180003d7c f   MSVCRT:utility.obj
 0001:00002db0       __scrt_dllmain_before_initialize_c 0000000180003db0 f   MSVCRT:utility.obj
 0001:00002dc8       __scrt_dllmain_crt_thread_attach 0000000180003dc8 f   MSVCRT:utility.obj
 0001:00002df0       __scrt_dllmain_crt_thread_detach 0000000180003df0 f   MSVCRT:utility.obj
 0001:00002e08       __scrt_dllmain_exception_filter 0000000180003e08 f   MSVCRT:utility.obj
 0001:00002e68       __scrt_dllmain_uninitialize_c 0000000180003e68 f   MSVCRT:utility.obj
 0001:00002e98       __scrt_dllmain_uninitialize_critical 0000000180003e98 f   MSVCRT:utility.obj
 0001:00002eac       __scrt_initialize_crt      0000000180003eac f   MSVCRT:utility.obj
 0001:00002ef8       __scrt_initialize_onexit_tables 0000000180003ef8 f   MSVCRT:utility.obj
 0001:00002f84       __scrt_is_nonwritable_in_current_image 0000000180003f84 f   MSVCRT:utility.obj
 0001:0000301c       __scrt_release_startup_lock 000000018000401c f   MSVCRT:utility.obj
 0001:00003040       __scrt_uninitialize_crt    0000000180004040 f   MSVCRT:utility.obj
 0001:0000306c       _onexit                    000000018000406c f   MSVCRT:utility.obj
 0001:000030a8       atexit                     00000001800040a8 f   MSVCRT:utility.obj
 0001:000030c0       __crt_debugger_hook        00000001800040c0 f   MSVCRT:utility_desktop.obj
 0001:000030c8       __scrt_fastfail            00000001800040c8 f   MSVCRT:utility_desktop.obj
 0001:00003214       _guard_check_icall_nop     0000000180004214 f i MSVCRT:guard_support.obj
 0001:00003218       __security_init_cookie     0000000180004218 f   MSVCRT:gs_support.obj
 0001:000032c4       DllMain                    00000001800042c4 f   MSVCRT:dll_dllmain_stub.obj
 0001:000032e8       ?__scrt_initialize_type_info@@YAXXZ 00000001800042e8 f   MSVCRT:tncleanup.obj
 0001:000032f8       ?__scrt_uninitialize_type_info@@YAXXZ 00000001800042f8 f   MSVCRT:tncleanup.obj
 0001:00003304       __local_stdio_scanf_options 0000000180004304 f i MSVCRT:default_local_stdio_options.obj
 0001:0000330c       __scrt_initialize_default_local_stdio_options 000000018000430c f   MSVCRT:default_local_stdio_options.obj
 0001:00003328       __scrt_get_dyn_tls_init_callback 0000000180004328 f   MSVCRT:dyn_tls_init.obj
 0001:00003330       _RTC_Initialize            0000000180004330 f   MSVCRT:initsect.obj
 0001:0000336c       _RTC_Terminate             000000018000436c f   MSVCRT:initsect.obj
 0001:000033a8       __isa_available_init       00000001800043a8 f   MSVCRT:cpu_disp.obj
 0001:00003554       _get_startup_argv_mode     0000000180004554 f   MSVCRT:argv_mode.obj
 0001:0000355c       __scrt_is_ucrt_dll_in_use  000000018000455c f   MSVCRT:ucrt_detection.obj
 0001:00003570       memcpy                     0000000180004570 f   vcruntime:VCRUNTIME140.dll
 0001:00003576       memset                     0000000180004576 f   vcruntime:VCRUNTIME140.dll
 0001:0000357c       strchr                     000000018000457c f   vcruntime:VCRUNTIME140.dll
 0001:00003582       __C_specific_handler       0000000180004582 f   vcruntime:VCRUNTIME140.dll
 0001:00003588       __std_type_info_destroy_list 0000000180004588 f   vcruntime:VCRUNTIME140.dll
 0001:0000358e       strcmp                     000000018000458e f   ucrt:api-ms-win-crt-string-l1-1-0.dll
 0001:00003594       strlen                     0000000180004594 f   ucrt:api-ms-win-crt-string-l1-1-0.dll
 0001:0000359a       _initterm                  000000018000459a f   ucrt:api-ms-win-crt-runtime-l1-1-0.dll
 0001:000035a0       _initterm_e                00000001800045a0 f   ucrt:api-ms-win-crt-runtime-l1-1-0.dll
 0001:000035a6       _seh_filter_dll            00000001800045a6 f   ucrt:api-ms-win-crt-runtime-l1-1-0.dll
 0001:000035ac       _configure_narrow_argv     00000001800045ac f   ucrt:api-ms-win-crt-runtime-l1-1-0.dll
 0001:000035b2       _initialize_narrow_environment 00000001800045b2 f   ucrt:api-ms-win-crt-runtime-l1-1-0.dll
 0001:000035b8       _initialize_onexit_table   00000001800045b8 f   ucrt:api-ms-win-crt-runtime-l1-1-0.dll
 0001:000035be       _register_onexit_function  00000001800045be f   ucrt:api-ms-win-crt-runtime-l1-1-0.dll
 0001:000035c4       _execute_onexit_table      00000001800045c4 f   ucrt:api-ms-win-crt-runtime-l1-1-0.dll
 0001:000035ca       _crt_atexit                00000001800045ca f   ucrt:api-ms-win-crt-runtime-l1-1-0.dll
 0001:000035d0       _cexit                     00000001800045d0 f   ucrt:api-ms-win-crt-runtime-l1-1-0.dll
 0001:000035d8       __acrt_initialize          00000001800045d8 f   MSVCRT:ucrt_stubs.obj
 0001:000035d8       __acrt_thread_attach       00000001800045d8 f   MSVCRT:ucrt_stubs.obj
 0001:000035d8       __acrt_thread_detach       00000001800045d8 f   MSVCRT:ucrt_stubs.obj
 0001:000035d8       __acrt_uninitialize        00000001800045d8 f   MSVCRT:ucrt_stubs.obj
 0001:000035d8       __acrt_uninitialize_critical 00000001800045d8 f   MSVCRT:ucrt_stubs.obj
 0001:000035d8       __scrt_stub_for_acrt_initialize 00000001800045d8 f   MSVCRT:ucrt_stubs.obj
 0001:000035d8       __scrt_stub_for_acrt_thread_attach 00000001800045d8 f   MSVCRT:ucrt_stubs.obj
 0001:000035d8       __scrt_stub_for_acrt_thread_detach 00000001800045d8 f   MSVCRT:ucrt_stubs.obj
 0001:000035d8       __scrt_stub_for_acrt_uninitialize 00000001800045d8 f   MSVCRT:ucrt_stubs.obj
 0001:000035d8       __scrt_stub_for_acrt_uninitialize_critical 00000001800045d8 f   MSVCRT:ucrt_stubs.obj
 0001:000035d8       __vcrt_initialize          00000001800045d8 f   MSVCRT:ucrt_stubs.obj
 0001:000035d8       __vcrt_thread_attach       00000001800045d8 f   MSVCRT:ucrt_stubs.obj
 0001:000035d8       __vcrt_thread_detach       00000001800045d8 f   MSVCRT:ucrt_stubs.obj
 0001:000035d8       __vcrt_uninitialize        00000001800045d8 f   MSVCRT:ucrt_stubs.obj
 0001:000035d8       __vcrt_uninitialize_critical 00000001800045d8 f   MSVCRT:ucrt_stubs.obj
 0001:000035dc       __scrt_stub_for_is_c_termination_complete 00000001800045dc f   MSVCRT:ucrt_stubs.obj
 0001:000035dc       _is_c_termination_complete 00000001800045dc f   MSVCRT:ucrt_stubs.obj
 0001:000035f0       _guard_dispatch_icall_nop  00000001800045f0 f   MSVCRT:guard_dispatch.obj
 0001:00003610       _guard_xfg_dispatch_icall_nop 0000000180004610 f   MSVCRT:guard_xfg_dispatch.obj
 0002:00000000       __imp_RtlCaptureContext    0000000180005000     kernel32:KERNEL32.dll
 0002:00000008       __imp_RtlLookupFunctionEntry 0000000180005008     kernel32:KERNEL32.dll
 0002:00000010       __imp_RtlVirtualUnwind     0000000180005010     kernel32:KERNEL32.dll
 0002:00000018       __imp_UnhandledExceptionFilter 0000000180005018     kernel32:KERNEL32.dll
 0002:00000020       __imp_SetUnhandledExceptionFilter 0000000180005020     kernel32:KERNEL32.dll
 0002:00000028       __imp_GetCurrentProcess    0000000180005028     kernel32:KERNEL32.dll
 0002:00000030       __imp_TerminateProcess     0000000180005030     kernel32:KERNEL32.dll
 0002:00000038       __imp_IsProcessorFeaturePresent 0000000180005038     kernel32:KERNEL32.dll
 0002:00000040       __imp_CloseHandle          0000000180005040     kernel32:KERNEL32.dll
 0002:00000048       __imp_InitializeCriticalSectionAndSpinCount 0000000180005048     kernel32:KERNEL32.dll
 0002:00000050       __imp_DeleteCriticalSection 0000000180005050     kernel32:KERNEL32.dll
 0002:00000058       __imp_CreateEventW         0000000180005058     kernel32:KERNEL32.dll
 0002:00000060       __imp_GetModuleHandleW     0000000180005060     kernel32:KERNEL32.dll
 0002:00000068       __imp_GetProcAddress       0000000180005068     kernel32:KERNEL32.dll
 0002:00000070       __imp_IsDebuggerPresent    0000000180005070     kernel32:KERNEL32.dll
 0002:00000078       __imp_QueryPerformanceCounter 0000000180005078     kernel32:KERNEL32.dll
 0002:00000080       __imp_GetCurrentProcessId  0000000180005080     kernel32:KERNEL32.dll
 0002:00000088       __imp_GetCurrentThreadId   0000000180005088     kernel32:KERNEL32.dll
 0002:00000090       __imp_GetSystemTimeAsFileTime 0000000180005090     kernel32:KERNEL32.dll
 0002:00000098       __imp_DisableThreadLibraryCalls 0000000180005098     kernel32:KERNEL32.dll
 0002:000000a0       __imp_InitializeSListHead  00000001800050a0     kernel32:KERNEL32.dll
 0002:000000a8       \177KERNEL32_NULL_THUNK_DATA 00000001800050a8     kernel32:KERNEL32.dll
 0002:000000b0       __imp_memcpy               00000001800050b0     vcruntime:VCRUNTIME140.dll
 0002:000000b8       __imp_memset               00000001800050b8     vcruntime:VCRUNTIME140.dll
 0002:000000c0       __imp_strchr               00000001800050c0     vcruntime:VCRUNTIME140.dll
 0002:000000c8       __imp___C_specific_handler 00000001800050c8     vcruntime:VCRUNTIME140.dll
 0002:000000d0       __imp___std_type_info_destroy_list 00000001800050d0     vcruntime:VCRUNTIME140.dll
 0002:000000d8       \177VCRUNTIME140_NULL_THUNK_DATA 00000001800050d8     vcruntime:VCRUNTIME140.dll
 0002:000000e0       __imp_strtol               00000001800050e0     ucrt:api-ms-win-crt-convert-l1-1-0.dll
 0002:000000e8       \177api-ms-win-crt-convert-l1-1-0_NULL_THUNK_DATA 00000001800050e8     ucrt:api-ms-win-crt-convert-l1-1-0.dll
 0002:000000f0       __imp_malloc               00000001800050f0     ucrt:api-ms-win-crt-heap-l1-1-0.dll
 0002:000000f8       __imp_free                 00000001800050f8     ucrt:api-ms-win-crt-heap-l1-1-0.dll
 0002:00000100       \177api-ms-win-crt-heap-l1-1-0_NULL_THUNK_DATA 0000000180005100     ucrt:api-ms-win-crt-heap-l1-1-0.dll
 0002:00000108       __imp__errno               0000000180005108     ucrt:api-ms-win-crt-runtime-l1-1-0.dll
 0002:00000110       __imp_exit                 0000000180005110     ucrt:api-ms-win-crt-runtime-l1-1-0.dll
 0002:00000118       __imp__cexit               0000000180005118     ucrt:api-ms-win-crt-runtime-l1-1-0.dll
 0002:00000120       __imp__crt_atexit          0000000180005120     ucrt:api-ms-win-crt-runtime-l1-1-0.dll
 0002:00000128       __imp__execute_onexit_table 0000000180005128     ucrt:api-ms-win-crt-runtime-l1-1-0.dll
 0002:00000130       __imp__register_onexit_function 0000000180005130     ucrt:api-ms-win-crt-runtime-l1-1-0.dll
 0002:00000138       __imp__initialize_onexit_table 0000000180005138     ucrt:api-ms-win-crt-runtime-l1-1-0.dll
 0002:00000140       __imp__initialize_narrow_environment 0000000180005140     ucrt:api-ms-win-crt-runtime-l1-1-0.dll
 0002:00000148       __imp__configure_narrow_argv 0000000180005148     ucrt:api-ms-win-crt-runtime-l1-1-0.dll
 0002:00000150       __imp__seh_filter_dll      0000000180005150     ucrt:api-ms-win-crt-runtime-l1-1-0.dll
 0002:00000158       __imp__initterm_e          0000000180005158     ucrt:api-ms-win-crt-runtime-l1-1-0.dll
 0002:00000160       __imp__initterm            0000000180005160     ucrt:api-ms-win-crt-runtime-l1-1-0.dll
 0002:00000168       \177api-ms-win-crt-runtime-l1-1-0_NULL_THUNK_DATA 0000000180005168     ucrt:api-ms-win-crt-runtime-l1-1-0.dll
 0002:00000170       __imp___acrt_iob_func      0000000180005170     ucrt:api-ms-win-crt-stdio-l1-1-0.dll
 0002:00000178       __imp_fflush               0000000180005178     ucrt:api-ms-win-crt-stdio-l1-1-0.dll
 0002:00000180       __imp___stdio_common_vsprintf 0000000180005180     ucrt:api-ms-win-crt-stdio-l1-1-0.dll
 0002:00000188       __imp___stdio_common_vfprintf 0000000180005188     ucrt:api-ms-win-crt-stdio-l1-1-0.dll
 0002:00000190       \177api-ms-win-crt-stdio-l1-1-0_NULL_THUNK_DATA 0000000180005190     ucrt:api-ms-win-crt-stdio-l1-1-0.dll
 0002:00000198       __imp_strcmp               0000000180005198     ucrt:api-ms-win-crt-string-l1-1-0.dll
 0002:000001a0       __imp__strdup              00000001800051a0     ucrt:api-ms-win-crt-string-l1-1-0.dll
 0002:000001a0       __imp_strdup               00000001800051a0     ucrt:api-ms-win-crt-string-l1-1-0.dll
 0002:000001a8       __imp_strlen               00000001800051a8     ucrt:api-ms-win-crt-string-l1-1-0.dll
 0002:000001b0       __imp_strpbrk              00000001800051b0     ucrt:api-ms-win-crt-string-l1-1-0.dll
 0002:000001b8       __imp_strncpy              00000001800051b8     ucrt:api-ms-win-crt-string-l1-1-0.dll
 0002:000001c0       \177api-ms-win-crt-string-l1-1-0_NULL_THUNK_DATA 00000001800051c0     ucrt:api-ms-win-crt-string-l1-1-0.dll
 0002:000001c8       __guard_check_icall_fptr   00000001800051c8     MSVCRT:guard_support.obj
 0002:000001d0       __guard_xfg_check_icall_fptr 00000001800051d0     MSVCRT:guard_support.obj
 0002:000001d8       __guard_dispatch_icall_fptr 00000001800051d8     MSVCRT:guard_support.obj
 0002:000001e0       __guard_xfg_dispatch_icall_fptr 00000001800051e0     MSVCRT:guard_support.obj
 0002:000001e8       __guard_xfg_table_dispatch_icall_fptr 00000001800051e8     MSVCRT:guard_support.obj
 0002:000001f0       __castguard_check_failure_os_handled_fptr 00000001800051f0     MSVCRT:guard_support.obj
 0002:000001f8       __guard_memcpy_fptr        00000001800051f8     vcruntime:softmemtag.obj
 0002:00000200       __xc_a                     0000000180005200     MSVCRT:initializers.obj
 0002:00000208       __xc_z                     0000000180005208     MSVCRT:initializers.obj
 0002:00000210       __xi_a                     0000000180005210     MSVCRT:initializers.obj
 0002:00000220       __xi_z                     0000000180005220     MSVCRT:initializers.obj
 0002:00000228       __xl_a                     0000000180005228     MSVCRT:tlssup.obj
 0002:00000230       __xl_z                     0000000180005230     MSVCRT:tlssup.obj
 0002:00000238       __xp_a                     0000000180005238     MSVCRT:initializers.obj
 0002:00000240       __xp_z                     0000000180005240     MSVCRT:initializers.obj
 0002:00000248       __xt_a                     0000000180005248     MSVCRT:initializers.obj
 0002:00000250       __xt_z                     0000000180005250     MSVCRT:initializers.obj
 0002:00000260       ??_C@_06FALKBLGB@?$DMinit?$DO@ 0000000180005260     liblocaltab005.obj
 0002:00000270       g_refKindStr               0000000180005270     liblocaltab005.obj
 0002:00000420       ??_C@_09BPLDFGCI@unknown_0@ 0000000180005420     liblocaltab005.obj
 0002:00000430       ??_C@_0BL@FPNMECJD@JVMTI_HEAP_REFERENCE_CLASS@ 0000000180005430     liblocaltab005.obj
 0002:00000450       ??_C@_0BL@FKGKKLNM@JVMTI_HEAP_REFERENCE_FIELD@ 0000000180005450     liblocaltab005.obj
 0002:00000470       ??_C@_0CD@CAEHCFJF@JVMTI_HEAP_REFERENCE_ARRAY_ELEM@ 0000000180005470     liblocaltab005.obj
 0002:00000498       ??_C@_0CC@DNEBMCNK@JVMTI_HEAP_REFERENCE_CLASS_LOAD@ 0000000180005498     liblocaltab005.obj
 0002:000004c0       ??_C@_0BN@CJMIPEBB@JVMTI_HEAP_REFERENCE_SIGNERS@ 00000001800054c0     liblocaltab005.obj
 0002:000004e0       ??_C@_0CH@HBOIDPEB@JVMTI_HEAP_REFERENCE_PROTECTION@ 00000001800054e0     liblocaltab005.obj
 0002:00000508       ??_C@_0BP@MDKGDGKL@JVMTI_HEAP_REFERENCE_INTERFACE@ 0000000180005508     liblocaltab005.obj
 0002:00000528       ??_C@_0CC@JJMIHNJH@JVMTI_HEAP_REFERENCE_STATIC_FIE@ 0000000180005528     liblocaltab005.obj
 0002:00000550       ??_C@_0CD@IDHEEGID@JVMTI_HEAP_REFERENCE_CONSTANT_P@ 0000000180005550     liblocaltab005.obj
 0002:00000578       ??_C@_0CA@EFFCHNG@JVMTI_HEAP_REFERENCE_SUPERCLASS@ 0000000180005578     liblocaltab005.obj
 0002:00000598       ??_C@_0L@PCDFHGCJ@unknown_11@ 0000000180005598     liblocaltab005.obj
 0002:000005a8       ??_C@_0L@NJBICFOK@unknown_12@ 00000001800055a8     liblocaltab005.obj
 0002:000005b8       ??_C@_0L@MAADBEKL@unknown_13@ 00000001800055b8     liblocaltab005.obj
 0002:000005c8       ??_C@_0L@IPECICGM@unknown_14@ 00000001800055c8     liblocaltab005.obj
 0002:000005d8       ??_C@_0L@JGFJLDCN@unknown_15@ 00000001800055d8     liblocaltab005.obj
 0002:000005e8       ??_C@_0L@LNHEOAOO@unknown_16@ 00000001800055e8     liblocaltab005.obj
 0002:000005f8       ??_C@_0L@KEGPNBKP@unknown_17@ 00000001800055f8     liblocaltab005.obj
 0002:00000608       ??_C@_0L@CDPHMNGA@unknown_18@ 0000000180005608     liblocaltab005.obj
 0002:00000618       ??_C@_0L@DKOMPMCB@unknown_19@ 0000000180005618     liblocaltab005.obj
 0002:00000628       ??_C@_0L@OJGIPJDB@unknown_20@ 0000000180005628     liblocaltab005.obj
 0002:00000638       ??_C@_0CA@KAOFNDEM@JVMTI_HEAP_REFERENCE_JNI_GLOBAL@ 0000000180005638     liblocaltab005.obj
 0002:00000658       ??_C@_0CC@HPFAJBK@JVMTI_HEAP_REFERENCE_SYSTEM_CLA@ 0000000180005658     liblocaltab005.obj
 0002:00000680       ??_C@_0BN@FDEGFOHC@JVMTI_HEAP_REFERENCE_MONITOR@ 0000000180005680     liblocaltab005.obj
 0002:000006a0       ??_C@_0CB@HKIBCMAJ@JVMTI_HEAP_REFERENCE_STACK_LOCA@ 00000001800056a0     liblocaltab005.obj
 0002:000006c8       ??_C@_0BP@EAACMMOE@JVMTI_HEAP_REFERENCE_JNI_LOCAL@ 00000001800056c8     liblocaltab005.obj
 0002:000006e8       ??_C@_0BM@IJDEOGOE@JVMTI_HEAP_REFERENCE_THREAD@ 00000001800056e8     liblocaltab005.obj
 0002:00000708       ??_C@_0BL@EDGPPKC@JVMTI_HEAP_REFERENCE_OTHER@ 0000000180005708     liblocaltab005.obj
 0002:00000724       ??_C@_04BCJPDBDA@Code@     0000000180005724     liblocaltab005.obj
 0002:00000730       ??_C@_0BA@OCLMCFKC@LineNumberTable@ 0000000180005730     liblocaltab005.obj
 0002:00000740       ??_C@_0BD@CPAEPILC@LocalVariableTable@ 0000000180005740     liblocaltab005.obj
 0002:00000758       ??_C@_0BH@NMBDNHBD@LocalVariableTypeTable@ 0000000180005758     liblocaltab005.obj
 0002:00000770       ??_C@_0O@HIHEEDNJ@StackMapTable@ 0000000180005770     liblocaltab005.obj
 0002:00000780       ??_C@_03GAEACAIP@?$CI?$CJV@ 0000000180005780     liblocaltab005.obj
 0002:00000784       ??_C@_04IIAJELJL@this@     0000000180005784     liblocaltab005.obj
 0002:00000790       ??_C@_0CP@GBBPGAIM@Lnsk?1jvmti?1GetLocalVariableTabl@ 0000000180005790     liblocaltab005.obj
 0002:000007c0       ??_C@_04MLLLIHIP@null@     00000001800057c0     liblocaltab005.obj
 0002:000007c8       ??_C@_08NOKDOCEA@constr_b@ 00000001800057c8     liblocaltab005.obj
 0002:000007d8       ??_C@_0CP@GDFJNONF@Lnsk?1jvmti?1GetLocalVariableTabl@ 00000001800057d8     liblocaltab005.obj
 0002:00000810       ??_C@_0ED@MJOLCBBL@Lnsk?1jvmti?1GetLocalVariableTabl@ 0000000180005810     liblocaltab005.obj
 0002:00000858       ??_C@_08DNFHDLIL@constr_i@ 0000000180005858     liblocaltab005.obj
 0002:00000864       ??_C@_01JPJNBJEM@I@        0000000180005864     liblocaltab005.obj
 0002:00000868       ??_C@_08MHLINDAB@constr_c@ 0000000180005868     liblocaltab005.obj
 0002:00000878       ??_C@_0CP@GCJLLEOC@Lnsk?1jvmti?1GetLocalVariableTabl@ 0000000180005878     liblocaltab005.obj
 0002:000008b0       ??_C@_0FH@MAMPHDHA@Lnsk?1jvmti?1GetLocalVariableTabl@ 00000001800058b0     liblocaltab005.obj
 0002:00000908       ??_C@_08LKMPCHEE@constr_f@ 0000000180005908     liblocaltab005.obj
 0002:00000914       ??_C@_01BIAFAFID@F@        0000000180005914     liblocaltab005.obj
 0002:00000918       ??_C@_09NKOEGJOK@constr_ch@ 0000000180005918     liblocaltab005.obj
 0002:00000924       ??_C@_01GFHCPBMG@C@        0000000180005924     liblocaltab005.obj
 0002:00000928       ??_C@_09EJPAMBLC@constr_if@ 0000000180005928     liblocaltab005.obj
 0002:00000938       ??_C@_0DA@HJANKKFP@Lnsk?1jvmti?1GetLocalVariableTabl@ 0000000180005938     liblocaltab005.obj
 0002:00000970       ??_C@_0EE@MPDKDEHM@Lnsk?1jvmti?1GetLocalVariableTabl@ 0000000180005970     liblocaltab005.obj
 0002:000009b4       ??_C@_05BHHOJHHJ@ins_c@    00000001800059b4     liblocaltab005.obj
 0002:000009bc       ??_C@_05ONJBHPPD@ins_i@    00000001800059bc     liblocaltab005.obj
 0002:000009c4       ??_C@_01LELAEKIP@J@        00000001800059c4     liblocaltab005.obj
 0002:000009c8       ??_C@_08JBHNCGHE@ltab005d@ 00000001800059c8     liblocaltab005.obj
 0002:000009d8       ??_C@_0CP@GHNEKCGH@Lnsk?1jvmti?1GetLocalVariableTabl@ 00000001800059d8     liblocaltab005.obj
 0002:00000a10       ??_C@_0ED@DFEJLHJK@Lnsk?1jvmti?1GetLocalVariableTabl@ 0000000180005a10     liblocaltab005.obj
 0002:00000a54       ??_C@_05NPKHBNHB@ins_k@    0000000180005a54     liblocaltab005.obj
 0002:00000a5c       ??_C@_05JAOGILLG@ins_l@    0000000180005a5c     liblocaltab005.obj
 0002:00000a64       ??_C@_05HDBCFCHN@ins_g@    0000000180005a64     liblocaltab005.obj
 0002:00000a70       ??_C@_0CP@GFJCBMDO@Lnsk?1jvmti?1GetLocalVariableTabl@ 0000000180005a70     liblocaltab005.obj
 0002:00000aa0       ??_C@_0FP@LJMKMFAH@Lnsk?1jvmti?1GetLocalVariableTabl@ 0000000180005aa0     liblocaltab005.obj
 0002:00000b00       ??_C@_06OPKJFGKF@stat_x@   0000000180005b00     liblocaltab005.obj
 0002:00000b08       ??_C@_06PGLCGHOE@stat_y@   0000000180005b08     liblocaltab005.obj
 0002:00000b10       ??_C@_06NNJPDECH@stat_z@   0000000180005b10     liblocaltab005.obj
 0002:00000b18       ??_C@_06JHFNCGHG@stat_j@   0000000180005b18     liblocaltab005.obj
 0002:00000b20       ??_C@_01CKDDGHAB@D@        0000000180005b20     liblocaltab005.obj
 0002:00000b24       ??_C@_06JNOALPI@stat_d@    0000000180005b24     liblocaltab005.obj
 0002:00000b30       ??_C@_0EB@NDDNNIJO@Lnsk?1jvmti?1GetLocalVariableTabl@ 0000000180005b30     liblocaltab005.obj
 0002:00000b78       ??_C@_09EKMGEFHL@insMethod@ 0000000180005b78     liblocaltab005.obj
 0002:00000b88       ??_C@_0DF@OADIMGG@?$CICJLnsk?1jvmti?1GetLocalVariableT@ 0000000180005b88     liblocaltab005.obj
 0002:00000bc0       ??_C@_0L@KCCHGEID@statMethod@ 0000000180005bc0     liblocaltab005.obj
 0002:00000bcc       ??_C@_06KGOANGDP@?$CIIII?$CJD@ 0000000180005bcc     liblocaltab005.obj
 0002:00000bd8       ??_C@_0L@HCDIAMJG@?9?5?$CFs?0?5?$CFd?3?5@ 0000000180005bd8     liblocaltab005.obj
 0002:00000bf0       ??_C@_0JI@HLPECLFI@?$CD?5?4?4?4?6?$CD?5ERROR?3?5too?5many?5complai@ 0000000180005bf0     liblocaltab005.obj
 0002:00000c90       ??_C@_0ED@JNEKCCOB@The?5following?5fake?5exception?5st@ 0000000180005c90     liblocaltab005.obj
 0002:00000cd8       ??_C@_0CN@FCNMDFBH@nsk?4share?4Fake_Exception_for_RU@ 0000000180005cd8     liblocaltab005.obj
 0002:00000d08       ??_C@_08PGFFNAEI@?$CI?$CFs?3?$CFd?$CJ?5@ 0000000180005d08     liblocaltab005.obj
 0002:00000d18       ??_C@_0DP@IENMAEGI@s?2test?2hotspot?2jtreg?2vmTestbase@ 0000000180005d18     liblocaltab005.obj
 0002:00000d58       ??_C@_0BL@NDJLFFJB@?7at?5nsk_lvcomplain?$CI?$CFs?3?$CFd?$CJ?6@ 0000000180005d58     liblocaltab005.obj
 0002:00000d78       ??_C@_0BC@JOOKAFKF@?$CD?5ERROR?3?5?$CFs?0?5?$CFd?3?5@ 0000000180005d78     liblocaltab005.obj
 0002:00000d90       ??_C@_09KJEAHMEH@?$CD?5ERROR?3?5@ 0000000180005d90     liblocaltab005.obj
 0002:00000d9c       ??_C@_02GPIOPFAK@?$DO?$DO@ 0000000180005d9c     liblocaltab005.obj
 0002:00000da0       ??_C@_02FODMEDOG@?$DM?$DM@ 0000000180005da0     liblocaltab005.obj
 0002:00000da4       ??_C@_02DJGKEECL@?4?4@     0000000180005da4     liblocaltab005.obj
 0002:00000da8       ??_C@_0O@CJPGJOAF@?9?5?$CFs?0?5?$CFd?3?5?$CFs?5@ 0000000180005da8     liblocaltab005.obj
 0002:00000db8       ??_C@_0CB@IAKPDOIC@?$CD?5?5?5verified?5assertion?5is?5FALSE@ 0000000180005db8     liblocaltab005.obj
 0002:00000de0       ??_C@_0CO@LGONDEPD@stdout?3?5fflush?5failed?5?9?5err?$DN?$CFd?5@ 0000000180005de0     liblocaltab005.obj
 0002:00000e10       ??_C@_0CO@KBGKJPBD@stderr?3?5fflush?5failed?5?9?5err?$DN?$CFd?5@ 0000000180005e10     liblocaltab005.obj
 0002:00000e40       ??_C@_01EEMJAFIK@?6@       0000000180005e40     liblocaltab005.obj
 0002:00000e48       ??_C@_0BB@JCNMKLLK@JVMTI_ERROR_NONE@ 0000000180005e48     liblocaltab005.obj
 0002:00000e60       ??_C@_0BL@LDIMKLPH@JVMTI_ERROR_INVALID_THREAD@ 0000000180005e60     liblocaltab005.obj
 0002:00000e80       ??_C@_0CB@PJFPAIKJ@JVMTI_ERROR_INVALID_THREAD_GROU@ 0000000180005e80     liblocaltab005.obj
 0002:00000ea8       ??_C@_0BN@LLMKHMNF@JVMTI_ERROR_INVALID_PRIORITY@ 0000000180005ea8     liblocaltab005.obj
 0002:00000ec8       ??_C@_0CB@MBOFKAGB@JVMTI_ERROR_THREAD_NOT_SUSPENDE@ 0000000180005ec8     liblocaltab005.obj
 0002:00000ef0       ??_C@_0BN@FABOLPBI@JVMTI_ERROR_THREAD_SUSPENDED@ 0000000180005ef0     liblocaltab005.obj
 0002:00000f10       ??_C@_0BN@FDGNOBJM@JVMTI_ERROR_THREAD_NOT_ALIVE@ 0000000180005f10     liblocaltab005.obj
 0002:00000f30       ??_C@_0BL@GOBIFKNJ@JVMTI_ERROR_INVALID_OBJECT@ 0000000180005f30     liblocaltab005.obj
 0002:00000f50       ??_C@_0BK@FCMAJPPC@JVMTI_ERROR_INVALID_CLASS@ 0000000180005f50     liblocaltab005.obj
 0002:00000f70       ??_C@_0BP@IKLLBKEB@JVMTI_ERROR_CLASS_NOT_PREPARED@ 0000000180005f70     liblocaltab005.obj
 0002:00000f90       ??_C@_0BN@KLPPLKG@JVMTI_ERROR_INVALID_METHODID@ 0000000180005f90     liblocaltab005.obj
 0002:00000fb0       ??_C@_0BN@BCEKOKND@JVMTI_ERROR_INVALID_LOCATION@ 0000000180005fb0     liblocaltab005.obj
 0002:00000fd0       ??_C@_0BM@DFDGPME@JVMTI_ERROR_INVALID_FIELDID@ 0000000180005fd0     liblocaltab005.obj
 0002:00000ff0       ??_C@_0BL@NELIEPEC@JVMTI_ERROR_NO_MORE_FRAMES@ 0000000180005ff0     liblocaltab005.obj
 0002:00001010       ??_C@_0BJ@BDBECFDM@JVMTI_ERROR_OPAQUE_FRAME@ 0000000180006010     liblocaltab005.obj
 0002:00001030       ??_C@_0BK@MIIFNLOB@JVMTI_ERROR_TYPE_MISMATCH@ 0000000180006030     liblocaltab005.obj
 0002:00001050       ??_C@_0BJ@HPCAOILC@JVMTI_ERROR_INVALID_SLOT@ 0000000180006050     liblocaltab005.obj
 0002:00001070       ??_C@_0BG@CHILOPNI@JVMTI_ERROR_DUPLICATE@ 0000000180006070     liblocaltab005.obj
 0002:00001088       ??_C@_0BG@DIEMLHKM@JVMTI_ERROR_NOT_FOUND@ 0000000180006088     liblocaltab005.obj
 0002:000010a0       ??_C@_0BM@NHMCKHOB@JVMTI_ERROR_INVALID_MONITOR@ 00000001800060a0     liblocaltab005.obj
 0002:000010c0       ??_C@_0BO@PPEDAJGL@JVMTI_ERROR_NOT_MONITOR_OWNER@ 00000001800060c0     liblocaltab005.obj
 0002:000010e0       ??_C@_0BG@FCAIPEID@JVMTI_ERROR_INTERRUPT@ 00000001800060e0     liblocaltab005.obj
 0002:000010f8       ??_C@_0CB@EGDBNKOI@JVMTI_ERROR_INVALID_CLASS_FORMA@ 00000001800060f8     liblocaltab005.obj
 0002:00001120       ??_C@_0CG@DGKOGIAL@JVMTI_ERROR_CIRCULAR_CLASS_DEFI@ 0000000180006120     liblocaltab005.obj
 0002:00001148       ??_C@_0BP@ICEALPKC@JVMTI_ERROR_FAILS_VERIFICATION@ 0000000180006148     liblocaltab005.obj
 0002:00001168       ??_C@_0DC@JDACLMIO@JVMTI_ERROR_UNSUPPORTED_REDEFIN@ 0000000180006168     liblocaltab005.obj
 0002:000011a0       ??_C@_0DE@GKDKNOMJ@JVMTI_ERROR_UNSUPPORTED_REDEFIN@ 00000001800061a0     liblocaltab005.obj
 0002:000011d8       ??_C@_0BO@LAFKIOG@JVMTI_ERROR_INVALID_TYPESTATE@ 00000001800061d8     liblocaltab005.obj
 0002:000011f8       ??_C@_0DH@INDGCLLB@JVMTI_ERROR_UNSUPPORTED_REDEFIN@ 00000001800061f8     liblocaltab005.obj
 0002:00001230       ??_C@_0DE@NHEOMMGI@JVMTI_ERROR_UNSUPPORTED_REDEFIN@ 0000000180006230     liblocaltab005.obj
 0002:00001268       ??_C@_0CA@EKPNJOEP@JVMTI_ERROR_UNSUPPORTED_VERSION@ 0000000180006268     liblocaltab005.obj
 0002:00001288       ??_C@_0BN@OFFMAHHL@JVMTI_ERROR_NAMES_DONT_MATCH@ 0000000180006288     liblocaltab005.obj
 0002:000012a8       ??_C@_0DN@HHBBLAKE@JVMTI_ERROR_UNSUPPORTED_REDEFIN@ 00000001800062a8     liblocaltab005.obj
 0002:000012e8       ??_C@_0DO@HMBGBGNA@JVMTI_ERROR_UNSUPPORTED_REDEFIN@ 00000001800062e8     liblocaltab005.obj
 0002:00001328       ??_C@_0BP@PBECGKHJ@JVMTI_ERROR_UNMODIFIABLE_CLASS@ 0000000180006328     liblocaltab005.obj
 0002:00001348       ??_C@_0BK@CANILEHF@JVMTI_ERROR_NOT_AVAILABLE@ 0000000180006348     liblocaltab005.obj
 0002:00001368       ??_C@_0CE@INJKMEFK@JVMTI_ERROR_MUST_POSSESS_CAPABI@ 0000000180006368     liblocaltab005.obj
 0002:00001390       ??_C@_0BJ@LBFPFPDM@JVMTI_ERROR_NULL_POINTER@ 0000000180006390     liblocaltab005.obj
 0002:000013b0       ??_C@_0BP@CHJPNNEM@JVMTI_ERROR_ABSENT_INFORMATION@ 00000001800063b0     liblocaltab005.obj
 0002:000013d0       ??_C@_0BP@OMFMNLC@JVMTI_ERROR_INVALID_EVENT_TYPE@ 00000001800063d0     liblocaltab005.obj
 0002:000013f0       ??_C@_0BN@BIBNPHHO@JVMTI_ERROR_ILLEGAL_ARGUMENT@ 00000001800063f0     liblocaltab005.obj
 0002:00001410       ??_C@_0BK@KKNDHDCE@JVMTI_ERROR_NATIVE_METHOD@ 0000000180006410     liblocaltab005.obj
 0002:00001430       ??_C@_0BK@PMKCFHAE@JVMTI_ERROR_OUT_OF_MEMORY@ 0000000180006430     liblocaltab005.obj
 0002:00001450       ??_C@_0BK@NNJBDMNB@JVMTI_ERROR_ACCESS_DENIED@ 0000000180006450     liblocaltab005.obj
 0002:00001470       ??_C@_0BI@GHECLMNC@JVMTI_ERROR_WRONG_PHASE@ 0000000180006470     liblocaltab005.obj
 0002:00001488       ??_C@_0BF@OLIHJOII@JVMTI_ERROR_INTERNAL@ 0000000180006488     liblocaltab005.obj
 0002:000014a0       ??_C@_0BO@EOHGKJHI@JVMTI_ERROR_UNATTACHED_THREAD@ 00000001800064a0     liblocaltab005.obj
 0002:000014c0       ??_C@_0CA@LKHFDACL@JVMTI_ERROR_INVALID_ENVIRONMENT@ 00000001800064c0     liblocaltab005.obj
 0002:000014e0       ??_C@_0BA@MMFHLOKK@?$DMunknown?5error?$DO@ 00000001800064e0     liblocaltab005.obj
 0002:000014f0       ??_C@_0CF@CBHOKDB@throwable?5?$DN?5jni?9?$DOExceptionOccur@ 00000001800064f0     liblocaltab005.obj
 0002:00001518       ??_C@_03OFAPEBGM@?$CFs?6@  0000000180006518     liblocaltab005.obj
 0002:00001520       ??_C@_0DM@LPIGEGNJ@s?2test?2hotspot?2jtreg?2vmTestbase@ 0000000180006520     liblocaltab005.obj
 0002:00001560       ??_C@_0CC@NFCNPEPK@Exception?5in?5JNI?5call?5?$CIcleared?$CJ@ 0000000180006560     liblocaltab005.obj
 0002:00001588       ??_C@_0BJ@IBAKFIKF@jni?9?$DOExceptionDescribe?$CI?$CJ@ 0000000180006588     liblocaltab005.obj
 0002:000015a8       ??_C@_0BG@GGKALKMH@jni?9?$DOExceptionClear?$CI?$CJ@ 00000001800065a8     liblocaltab005.obj
 0002:000015c0       ??_C@_0CF@JMGFGJLJ@?$CD?5?5?5verified?5JNI?5assertion?5is?5F@ 00000001800065c0     liblocaltab005.obj
 0002:000015e8       ??_C@_07KBAMPNJK@verbose@  00000001800065e8     liblocaltab005.obj
 0002:000015f0       ??_C@_0DN@PKJBOLAP@nsk_jvmti_parseOptions?$CI?$CJ?3?5unexp@ 00000001800065f0     liblocaltab005.obj
 0002:00001630       ??_C@_05IMBNNINJ@trace@    0000000180006630     liblocaltab005.obj
 0002:00001638       ??_C@_0DD@BJKGNDMB@nsk_jvmti_parseOptions?$CI?$CJ?3?5no?5va@ 0000000180006638     liblocaltab005.obj
 0002:0000166c       ??_C@_04CGFJFPFD@none@     000000018000666c     liblocaltab005.obj
 0002:00001674       ??_C@_06BMELKFMA@before@   0000000180006674     liblocaltab005.obj
 0002:0000167c       ??_C@_05CMKPCFDK@after@    000000018000667c     liblocaltab005.obj
 0002:00001684       ??_C@_03NFKEKGGK@all@      0000000180006684     liblocaltab005.obj
 0002:00001688       ??_C@_0DM@NDNJGJKE@nsk_jvmti_parseOptions?$CI?$CJ?3?5uexpe@ 0000000180006688     liblocaltab005.obj
 0002:000016c8       ??_C@_08NBBJKJO@waittime@  00000001800066c8     liblocaltab005.obj
 0002:000016d8       ??_C@_0DO@CMHGAOHC@nsk_jvmti_parseOptions?$CI?$CJ?3?5not?5i@ 00000001800066d8     liblocaltab005.obj
 0002:00001718       ??_C@_0DL@LNMPBDLN@nsk_jvmti_parseOptions?$CI?$CJ?3?5negat@ 0000000180006718     liblocaltab005.obj
 0002:00001758       ??_C@_0DA@GMFJNOJH@nsk_jvmti_parseOptions?$CI?$CJ?3?5unkno@ 0000000180006758     liblocaltab005.obj
 0002:00001788       ??_C@_0CO@CCIAMEAN@nsk_jvmti_parseOptions?$CI?$CJ?3?5found@ 0000000180006788     liblocaltab005.obj
 0002:000017b8       ??_C@_0CJ@OEGPCGDL@nsk_jvmti_parseOptions?$CI?$CJ?3?5out?5o@ 00000001800067b8     liblocaltab005.obj
 0002:000017e8       ??_C@_0DI@NMBHPGGF@nsk_jvmti_parseOptions?$CI?$CJ?3?5too?5m@ 00000001800067e8     liblocaltab005.obj
 0002:00001820       ??_C@_03POGCGECB@?5?0?$HO@ 0000000180006820     liblocaltab005.obj
 0002:00001828       ??_C@_0CB@MLNJNCLJ@?5?5jvmti?5error?3?5code?$DN?$CFd?0?5name?$DN?$CFs@ 0000000180006828     liblocaltab005.obj
 0002:00001850       ??_C@_0CD@OHBGDKMK@?$CD?5?5?5jvmti?5error?3?5code?$DN?$CFd?0?5name?$DN@ 0000000180006850     liblocaltab005.obj
 0002:00001878       ??_C@_0CG@JNNCGPHB@?$CD?5?5?5error?5expected?3?5code?$DN?$CFd?0?5na@ 0000000180006878     liblocaltab005.obj
 0002:000018a0       ??_C@_0EB@IMGKPCGE@?$CIstr_obj?5?$DN?5jni?9?$DONewStringUTF?$CIco@ 00000001800068a0     liblocaltab005.obj
 0002:000018f0       ??_C@_0EA@HFOGGBCC@s?2test?2hotspot?2jtreg?2vmTestbase@ 00000001800068f0     liblocaltab005.obj
 0002:00001930       ??_C@_05KKCIMGE@error@     0000000180006930     liblocaltab005.obj
 0002:00001938       ??_C@_0CJ@JACLEAA@Test?5failed?5by?5setFailStatus?$CI?$CJ?4@ 0000000180006938     liblocaltab005.obj
 0002:00001968       ??_C@_0BD@HGNAOMCP@agent_data_monitor@ 0000000180006968     liblocaltab005.obj
 0002:00001980       ??_C@_0EB@OGCLGKLN@javaVM?9?$DOGetEnv?$CI?$CIvoid?5?$CK?$CK?$CJ?$CGjvmti_@ 0000000180006980     liblocaltab005.obj
 0002:000019d0       ??_C@_0EA@PNBCDMOA@s?2test?2hotspot?2jtreg?2vmTestbase@ 00000001800069d0     liblocaltab005.obj
 0002:00001a10       ??_C@_0CI@DDPIFBGM@init_agent_data?$CIjvmti_env?0?5?$CGage@ 0000000180006a10     liblocaltab005.obj
 0002:00001a38       ??_C@_0DI@ILAHDLMP@?$CI?$CKagentThreadProc?$CJ?$CIjvmti_env?0?5a@ 0000000180006a38     liblocaltab005.obj
 0002:00001a70       ??_C@_0BD@KDBALNLB@JVMTI?5agent?5thread@ 0000000180006a70     liblocaltab005.obj
 0002:00001a88       ??_C@_0BB@NOKBFPFO@java?1lang?1Thread@ 0000000180006a88     liblocaltab005.obj
 0002:00001aa0       ??_C@_0BG@IKDDPPGD@?$CILjava?1lang?1String?$DL?$CJV@ 0000000180006aa0     liblocaltab005.obj
 0002:00001ac0       ??_C@_0EB@IFJBFEKC@?$CIthreadClass?5?$DN?5jni_env?9?$DOFindCla@ 0000000180006ac0     liblocaltab005.obj
 0002:00001b10       ??_C@_0GF@FGFIBKKL@?$CIthreadCtor?5?$DN?5jni_env?9?$DOGetMetho@ 0000000180006b10     liblocaltab005.obj
 0002:00001b78       ??_C@_0DN@NCPDJLOG@?$CIthreadName?5?$DN?5jni_env?9?$DONewStrin@ 0000000180006b78     liblocaltab005.obj
 0002:00001bc0       ??_C@_0FE@PFKODBGC@?$CIthreadObject?5?$DN?5jni_env?9?$DONewObj@ 0000000180006bc0     liblocaltab005.obj
 0002:00001c20       ??_C@_0ED@HOBAHHJI@?$CIthreadGlobalRef?5?$DN?5jni_env?9?$DONew@ 0000000180006c20     liblocaltab005.obj
 0002:00001c70       ??_C@_0FN@HNJJAHFC@jvmti_env?9?$DORunAgentThread?$CIagent@ 0000000180006c70     liblocaltab005.obj
 0002:00001cd0       ??_C@_0EA@MOJDNKDF@Debuggee?5status?5sync?5aborted?5be@ 0000000180006cd0     liblocaltab005.obj
 0002:00001d10       ??_C@_0EA@EEOEJAEN@status?5?$DN?5syncDebuggeeStatus?$CIjni@ 0000000180006d10     liblocaltab005.obj
 0002:00001d50       ??_C@_0BL@JBCFNBMB@nsk_jvmti_resetAgentData?$CI?$CJ@ 0000000180006d50     liblocaltab005.obj
 0002:00001d70       ??_C@_0EL@LPBEELIP@s?2test?2hotspot?2jtreg?2vmTestbase@ 0000000180006d70     liblocaltab005.obj
 0002:00001dc0       ??_C@_0CK@JDAMFDMJ@jvmti?9?$DOSetTag?$CIo?0?5tag?$CJ?5?$DN?$DN?5JVMTI_@ 0000000180006dc0     liblocaltab005.obj
 0002:00001df0       ??_C@_0CC@DAMNHKNI@Can?8t?5set?5tag?5?$CFli?5for?5object?5?$CFl@ 0000000180006df0     liblocaltab005.obj
 0002:00001e18       ??_C@_0DL@HAJPNKEF@jvmti?9?$DOGetObjectHashCode?$CIo?0?5?$CGha@ 0000000180006e18     liblocaltab005.obj
 0002:00001e58       ??_C@_0BL@JFPIEOBF@Can?8t?5get?5hash?5object?5?$CFlx?6@ 0000000180006e58     liblocaltab005.obj
 0002:00001e78       ??_C@_0BG@DICPHBKN@setTag?3?5?$CF08x?5?$DM?9?5?$CF?53li@ 0000000180006e78     liblocaltab005.obj
 0002:00001e90       ??_C@_0DH@FCEEBDMJ@?$CIs?5?$DN?5jni?9?$DOGetStringUTFChars?$CIsIn@ 0000000180006e90     liblocaltab005.obj
 0002:00001ec8       ??_C@_0BJ@OKKGHDCN@Can?8t?5get?5string?5at?5?$CF?$CDp?6@ 0000000180006ec8     liblocaltab005.obj
 0002:00001ee8       ??_C@_0BP@EKFLGGFJ@Can?8t?5get?5string?5at?5?$CF?$CDp?3?5null?6@ 0000000180006ee8     liblocaltab005.obj
 0002:00001f08       ??_C@_06ICODBHCL@?5?1?1?5?$CFs@ 0000000180006f08     liblocaltab005.obj
 0002:00001f10       ??_C@_0DB@KGFPLEGO@?$CIr?5?$DN?5jvmti?9?$DOGetTag?$CIo?0?5?$CGtag?$CJ?$CJ?5?$DN?$DN@ 0000000180006f10     liblocaltab005.obj
 0002:00001f48       ??_C@_0CO@PDAGBCGJ@Can?8t?5GetTag?5for?5object?5?$CFlx?4?5Re@ 0000000180006f48     liblocaltab005.obj
 0002:00001f78       ??_C@_0CH@HPEODOHC@TEST_BUG?3?5Max?4?5number?5of?5refs?5r@ 0000000180006f78     liblocaltab005.obj
 0002:00001fa0       ??_C@_0DI@PHFCABIM@?$CIr?5?$DN?5jvmti?9?$DOGetTag?$CIfrom?0?5?$CGtagFr@ 0000000180006fa0     liblocaltab005.obj
 0002:00001fd8       ??_C@_0DI@MDEGFNKD@TEST_BUG?3?5Can?8t?5GetTag?5for?5obje@ 0000000180006fd8     liblocaltab005.obj
 0002:00002010       ??_C@_0DE@MLELJAHM@?$CIr?5?$DN?5jvmti?9?$DOGetTag?$CIto?0?5?$CGtagTo?$CJ?$CJ@ 0000000180007010     liblocaltab005.obj
 0002:00002048       ??_C@_08EMNENPBA@instance@ 0000000180007048     liblocaltab005.obj
 0002:00002054       ??_C@_06GGHJAEBN@static@   0000000180007054     liblocaltab005.obj
 0002:00002060       ??_C@_0FD@CNINKOKC@TEST?5FAILURE?3?5unable?5to?5get?5the@ 0000000180007060     liblocaltab005.obj
 0002:000020c0       ??_C@_0FM@PODFNKGD@s?2test?2hotspot?2jtreg?2vmTestbase@ 00000001800070c0     liblocaltab005.obj
 0002:00002120       ??_C@_0EB@LBJDHPCE@jvmti?9?$DOGetLocalVariableTable?$CIme@ 0000000180007120     liblocaltab005.obj
 0002:00002170       ??_C@_0FK@DPAEOJKF@TEST?5FAILED?3?5unable?5to?5get?5loca@ 0000000180007170     liblocaltab005.obj
 0002:000021d0       ??_C@_0HO@GLCJLICD@TEST?5FAILED?3?5?$CFs?5method?5?$CC?$CFs?$CC?0?5si@ 00000001800071d0     liblocaltab005.obj
 0002:00002250       ??_C@_0DL@IFPCNKCM@?7?$CFd?$CJ?5name?3?5?$CC?$CFs?$CC?6?7signature?3?5?$CC?$CFs@ 0000000180007250     liblocaltab005.obj
 0002:00002290       ??_C@_0HB@LGAEIHFG@?$DO?$DO?$DO?5Checking?5vars?5in?5the?5LocalV@ 0000000180007290     liblocaltab005.obj
 0002:00002310       ??_C@_0HD@OOOBBFGL@TEST?5FAILED?3?5?$CFs?5method?3?5?$CC?$CFs?$CC?5?$CC?$CF@ 0000000180007310     liblocaltab005.obj
 0002:00002390       ??_C@_0EF@MCOPBNJL@CHECK?5PASSED?3?5var?3?5?$CC?$CFs?$CC?0?6?7signa@ 0000000180007390     liblocaltab005.obj
 0002:000023d8       ??_C@_0CP@COGMBKNO@Deallocating?5the?5local?5variable@ 00000001800073d8     liblocaltab005.obj
 0002:00002408       ??_C@_0CN@BDGOOHFF@jvmti?9?$DODeallocate?$CI?$CIunsigned?5cha@ 0000000180007408     liblocaltab005.obj
 0002:00002438       ??_C@_04DAGPOOAC@?$DM?$DM?$DM?6@ 0000000180007438     liblocaltab005.obj
 0002:00002440       ??_C@_0CA@MNKGCBCG@nsk_jvmti_parseOptions?$CIoptions?$CJ@ 0000000180007440     liblocaltab005.obj
 0002:00002460       ??_C@_0DN@MIAMNFPH@?$CIjvmti?5?$DN?5nsk_jvmti_createJVMTIE@ 0000000180007460     liblocaltab005.obj
 0002:000024a0       ??_C@_0BO@DBKDIPGD@jvmti?9?$DOAddCapabilities?$CI?$CGcaps?$CJ@ 00000001800074a0     liblocaltab005.obj
 0002:000024c0       ??_C@_0BO@IAKFILDF@jvmti?9?$DOGetCapabilities?$CI?$CGcaps?$CJ@ 00000001800074c0     liblocaltab005.obj
 0002:000024e0       ??_C@_0DH@IJEIPLEC@Warning?3?5access?5to?5local?5variab@ 00000001800074e0     liblocaltab005.obj
 0002:00002530       ??_C@_1EC@JIJBPKFM@?$AAa?$AAp?$AAi?$AA?9?$AAm?$AAs?$AA?9?$AAw?$AAi?$AAn?$AA?9?$AAc?$AAo?$AAr?$AAe@ 0000000180007530     MSVCRT:thread_safe_statics.obj
 0002:00002578       ??_C@_1BK@MGMFAEKH@?$AAk?$AAe?$AAr?$AAn?$AAe?$AAl?$AA3?$AA2?$AA?4?$AAd?$AAl?$AAl@ 0000000180007578     MSVCRT:thread_safe_statics.obj
 0002:00002598       ??_C@_0BJ@JEBJOJFJ@SleepConditionVariableCS@ 0000000180007598     MSVCRT:thread_safe_statics.obj
 0002:000025b8       ??_C@_0BJ@PGPPEPCC@WakeAllConditionVariable@ 00000001800075b8     MSVCRT:thread_safe_statics.obj
 0002:000025d8       _pDefaultRawDllMain        00000001800075d8     MSVCRT:dll_dllmain.obj
 0002:000025d8       _pRawDllMain               00000001800075d8     MSVCRT:dll_dllmain.obj
 0002:000025e0       __xmm@ffffffffffffffffffffffffffffffff 00000001800075e0     MSVCRT:utility.obj
 0002:000025f0       _load_config_used          00000001800075f0     MSVCRT:loadcfg.obj
 0002:00002800       _tls_used                  0000000180007800     MSVCRT:tlssup.obj
 0002:00002828       __volatile_metadata        0000000180007828     <linker-defined>
 0002:00002be8       __rtc_iaa                  0000000180007be8     MSVCRT:initsect.obj
 0002:00002bf0       __rtc_izz                  0000000180007bf0     MSVCRT:initsect.obj
 0002:00002bf8       __rtc_taa                  0000000180007bf8     MSVCRT:initsect.obj
 0002:00002c00       __rtc_tzz                  0000000180007c00     MSVCRT:initsect.obj
 0002:00002c08       _tls_start                 0000000180007c08     MSVCRT:tlssup.obj
 0002:00002c0c       _Init_thread_epoch         0000000180007c0c     MSVCRT:thread_safe_statics.obj
 0002:00002c10       _tls_end                   0000000180007c10     MSVCRT:tlssup.obj
 0002:000032d4       __IMPORT_DESCRIPTOR_KERNEL32 00000001800082d4     kernel32:KERNEL32.dll
 0002:000032e8       __IMPORT_DESCRIPTOR_VCRUNTIME140 00000001800082e8     vcruntime:VCRUNTIME140.dll
 0002:000032fc       __IMPORT_DESCRIPTOR_api-ms-win-crt-heap-l1-1-0 00000001800082fc     ucrt:api-ms-win-crt-heap-l1-1-0.dll
 0002:00003310       __IMPORT_DESCRIPTOR_api-ms-win-crt-runtime-l1-1-0 0000000180008310     ucrt:api-ms-win-crt-runtime-l1-1-0.dll
 0002:00003324       __IMPORT_DESCRIPTOR_api-ms-win-crt-convert-l1-1-0 0000000180008324     ucrt:api-ms-win-crt-convert-l1-1-0.dll
 0002:00003338       __IMPORT_DESCRIPTOR_api-ms-win-crt-stdio-l1-1-0 0000000180008338     ucrt:api-ms-win-crt-stdio-l1-1-0.dll
 0002:0000334c       __IMPORT_DESCRIPTOR_api-ms-win-crt-string-l1-1-0 000000018000834c     ucrt:api-ms-win-crt-string-l1-1-0.dll
 0002:00003360       __NULL_IMPORT_DESCRIPTOR   0000000180008360     kernel32:KERNEL32.dll
 0003:000002a0       _Init_global_epoch         00000001800092a0     MSVCRT:thread_safe_statics.obj
 0003:000002b0       __security_cookie          00000001800092b0     MSVCRT:gs_cookie.obj
 0003:000002b8       __security_cookie_complement 00000001800092b8     MSVCRT:gs_cookie.obj
 0003:000002c0       __scrt_native_dllmain_reason 00000001800092c0     MSVCRT:utility.obj
 0003:000002c8       __isa_available            00000001800092c8     MSVCRT:cpu_disp.obj
 0003:000002cc       __isa_enabled              00000001800092cc     MSVCRT:cpu_disp.obj
 0003:000002d0       __memset_fast_string_threshold 00000001800092d0     MSVCRT:cpu_disp.obj
 0003:000002d8       __memset_nt_threshold      00000001800092d8     MSVCRT:cpu_disp.obj
 0003:000002e0       __scrt_ucrt_dll_is_in_use  00000001800092e0     MSVCRT:ucrt_stubs.obj
 0003:000002f0       g_wrongHeapCallbacks       00000001800092f0     liblocaltab005.obj
 0003:00000370       g_szTagInfo                0000000180009370     liblocaltab005.obj
 0003:000022b0       g_tagFlags                 000000018000b2b0     liblocaltab005.obj
 0003:00002698       g_refsToVerifyCnt          000000018000b698     liblocaltab005.obj
 0003:0000269c       g_fakeUserData             000000018000b69c     liblocaltab005.obj
 0003:000026a0       g_tagVisitCount            000000018000b6a0     liblocaltab005.obj
 0003:00003640       g_refsToVerify             000000018000c640     liblocaltab005.obj
 0003:0001ad40       g_userDataError            0000000180023d40     liblocaltab005.obj
 0003:0001aef0       ?_OptionsStorage@?1??__local_stdio_printf_options@@9@4_KA 0000000180023ef0     liblocaltab005.obj
 0003:0001b4b8       _tls_index                 00000001800244b8     MSVCRT:tlssup.obj
 0003:0001b4c0       __scrt_current_native_startup_state 00000001800244c0     MSVCRT:utility.obj
 0003:0001b4c8       __scrt_native_startup_lock 00000001800244c8     MSVCRT:utility.obj
 0003:0001b508       __scrt_debugger_hook_flag  0000000180024508     MSVCRT:utility_desktop.obj
 0003:0001b510       ?__type_info_root_node@@3U__type_info_node@@A 0000000180024510     MSVCRT:tncleanup.obj
 0003:0001b520       ?_OptionsStorage@?1??__local_stdio_scanf_options@@9@4_KA 0000000180024520     MSVCRT:default_local_stdio_options.obj
 0003:0001b528       __favor                    0000000180024528     MSVCRT:cpu_disp.obj
 0003:0001b530       __dyn_tls_init_callback    0000000180024530     <common>

 entry point at        0001:00002d00

 Static symbols

 0000:fffd9000       .debug$S                   0000000180000000     localtab005.exp
 0000:fffd9000       .debug$S                   0000000180000000     vcruntime:VCRUNTIME140.dll
 0000:fffd9000       .debug$S                   0000000180000000     vcruntime:VCRUNTIME140.dll
 0000:fffd9000       .debug$S                   0000000180000000     vcruntime:VCRUNTIME140.dll
 0000:fffd9000       .debug$S                   0000000180000000     vcruntime:VCRUNTIME140.dll
 0000:fffd9000       .debug$S                   0000000180000000     vcruntime:VCRUNTIME140.dll
 0000:fffd9000       .debug$S                   0000000180000000     vcruntime:VCRUNTIME140.dll
 0000:fffd9000       .debug$S                   0000000180000000     vcruntime:VCRUNTIME140.dll
 0000:fffd9000       .debug$S                   0000000180000000     ucrt:api-ms-win-crt-convert-l1-1-0.dll
 0000:fffd9000       .debug$S                   0000000180000000     ucrt:api-ms-win-crt-heap-l1-1-0.dll
 0000:fffd9000       .debug$S                   0000000180000000     ucrt:api-ms-win-crt-heap-l1-1-0.dll
 0000:fffd9000       .debug$S                   0000000180000000     ucrt:api-ms-win-crt-heap-l1-1-0.dll
 0000:fffd9000       .debug$S                   0000000180000000     ucrt:api-ms-win-crt-heap-l1-1-0.dll
 0000:fffd9000       .debug$S                   0000000180000000     ucrt:api-ms-win-crt-runtime-l1-1-0.dll
 0000:fffd9000       .debug$S                   0000000180000000     ucrt:api-ms-win-crt-runtime-l1-1-0.dll
 0000:fffd9000       .debug$S                   0000000180000000     ucrt:api-ms-win-crt-runtime-l1-1-0.dll
 0000:fffd9000       .debug$S                   0000000180000000     ucrt:api-ms-win-crt-runtime-l1-1-0.dll
 0000:fffd9000       .debug$S                   0000000180000000     ucrt:api-ms-win-crt-runtime-l1-1-0.dll
 0000:fffd9000       .debug$S                   0000000180000000     ucrt:api-ms-win-crt-runtime-l1-1-0.dll
 0000:fffd9000       .debug$S                   0000000180000000     ucrt:api-ms-win-crt-runtime-l1-1-0.dll
 0000:fffd9000       .debug$S                   0000000180000000     ucrt:api-ms-win-crt-runtime-l1-1-0.dll
 0000:fffd9000       .debug$S                   0000000180000000     ucrt:api-ms-win-crt-runtime-l1-1-0.dll
 0000:fffd9000       .debug$S                   0000000180000000     ucrt:api-ms-win-crt-runtime-l1-1-0.dll
 0000:fffd9000       .debug$S                   0000000180000000     ucrt:api-ms-win-crt-runtime-l1-1-0.dll
 0000:fffd9000       .debug$S                   0000000180000000     ucrt:api-ms-win-crt-runtime-l1-1-0.dll
 0000:fffd9000       .debug$S                   0000000180000000     ucrt:api-ms-win-crt-runtime-l1-1-0.dll
 0000:fffd9000       .debug$S                   0000000180000000     ucrt:api-ms-win-crt-runtime-l1-1-0.dll
 0000:fffd9000       .debug$S                   0000000180000000     ucrt:api-ms-win-crt-runtime-l1-1-0.dll
 0000:fffd9000       .debug$S                   0000000180000000     ucrt:api-ms-win-crt-runtime-l1-1-0.dll
 0000:fffd9000       .debug$S                   0000000180000000     ucrt:api-ms-win-crt-stdio-l1-1-0.dll
 0000:fffd9000       .debug$S                   0000000180000000     ucrt:api-ms-win-crt-stdio-l1-1-0.dll
 0000:fffd9000       .debug$S                   0000000180000000     ucrt:api-ms-win-crt-stdio-l1-1-0.dll
 0000:fffd9000       .debug$S                   0000000180000000     ucrt:api-ms-win-crt-stdio-l1-1-0.dll
 0000:fffd9000       .debug$S                   0000000180000000     ucrt:api-ms-win-crt-stdio-l1-1-0.dll
 0000:fffd9000       .debug$S                   0000000180000000     ucrt:api-ms-win-crt-stdio-l1-1-0.dll
 0000:fffd9000       .debug$S                   0000000180000000     ucrt:api-ms-win-crt-stdio-l1-1-0.dll
 0000:fffd9000       .debug$S                   0000000180000000     ucrt:api-ms-win-crt-stdio-l1-1-0.dll
 0000:fffd9000       .debug$S                   0000000180000000     ucrt:api-ms-win-crt-stdio-l1-1-0.dll
 0000:fffd9000       .debug$S                   0000000180000000     ucrt:api-ms-win-crt-stdio-l1-1-0.dll
 0000:fffd9000       .debug$S                   0000000180000000     ucrt:api-ms-win-crt-string-l1-1-0.dll
 0000:fffd9000       .debug$S                   0000000180000000     ucrt:api-ms-win-crt-string-l1-1-0.dll
 0000:fffd9000       .debug$S                   0000000180000000     ucrt:api-ms-win-crt-string-l1-1-0.dll
 0000:fffd9000       .debug$S                   0000000180000000     ucrt:api-ms-win-crt-string-l1-1-0.dll
 0000:fffd9000       .debug$S                   0000000180000000     ucrt:api-ms-win-crt-string-l1-1-0.dll
 0000:fffd9000       .debug$S                   0000000180000000     ucrt:api-ms-win-crt-string-l1-1-0.dll
 0000:fffd9000       .debug$S                   0000000180000000     ucrt:api-ms-win-crt-string-l1-1-0.dll
 0000:fffd9000       .debug$S                   0000000180000000     ucrt:api-ms-win-crt-string-l1-1-0.dll
 0000:fffd9000       .debug$S                   0000000180000000     kernel32:KERNEL32.dll
 0000:fffd9000       .debug$S                   0000000180000000     kernel32:KERNEL32.dll
 0000:fffd9000       .debug$S                   0000000180000000     kernel32:KERNEL32.dll
 0000:fffd9000       .debug$S                   0000000180000000     kernel32:KERNEL32.dll
 0000:fffd9000       .debug$S                   0000000180000000     kernel32:KERNEL32.dll
 0000:fffd9000       .debug$S                   0000000180000000     kernel32:KERNEL32.dll
 0000:fffd9000       .debug$S                   0000000180000000     kernel32:KERNEL32.dll
 0000:fffd9000       .debug$S                   0000000180000000     kernel32:KERNEL32.dll
 0000:fffd9000       .debug$S                   0000000180000000     kernel32:KERNEL32.dll
 0000:fffd9000       .debug$S                   0000000180000000     kernel32:KERNEL32.dll
 0000:fffd9000       .debug$S                   0000000180000000     kernel32:KERNEL32.dll
 0000:fffd9000       .debug$S                   0000000180000000     kernel32:KERNEL32.dll
 0000:fffd9000       .debug$S                   0000000180000000     kernel32:KERNEL32.dll
 0000:fffd9000       .debug$S                   0000000180000000     kernel32:KERNEL32.dll
 0000:fffd9000       .debug$S                   0000000180000000     kernel32:KERNEL32.dll
 0000:fffd9000       .debug$S                   0000000180000000     kernel32:KERNEL32.dll
 0000:fffd9000       .debug$S                   0000000180000000     kernel32:KERNEL32.dll
 0000:fffd9000       .debug$S                   0000000180000000     kernel32:KERNEL32.dll
 0000:fffd9000       .debug$S                   0000000180000000     kernel32:KERNEL32.dll
 0000:fffd9000       .debug$S                   0000000180000000     kernel32:KERNEL32.dll
 0000:fffd9000       .debug$S                   0000000180000000     kernel32:KERNEL32.dll
 0000:fffd9000       .debug$S                   0000000180000000     kernel32:KERNEL32.dll
 0000:fffd9000       .debug$S                   0000000180000000     kernel32:KERNEL32.dll
 0000:fffd9000       .debug$S                   0000000180000000     kernel32:KERNEL32.dll
 0000:fffd9000       .debug$S                   0000000180000000     kernel32:KERNEL32.dll
 0000:fffd9000       .debug$S                   0000000180000000     kernel32:KERNEL32.dll
 0000:fffd9000       .debug$S                   0000000180000000     kernel32:KERNEL32.dll
 0000:fffd9000       .debug$S                   0000000180000000     kernel32:KERNEL32.dll
 0001:00000ea0       addRefToVerify             0000000180001ea0 f   liblocaltab005.obj
 0001:00000f0c       agentThreadWrapper         0000000180001f0c f   liblocaltab005.obj
 0001:00001078       checkAttr                  0000000180002078 f   liblocaltab005.obj
 0001:00001588       check_option               0000000180002588 f   liblocaltab005.obj
 0001:000017d0       file_basename              00000001800027d0 f   liblocaltab005.obj
 0001:000021e8       startAgentThreadWrapper    00000001800031e8 f   liblocaltab005.obj
 0001:00002528       syncDebuggeeStatus         0000000180003528 f   liblocaltab005.obj
 0001:000027c8       capture_previous_context   00000001800037c8 f   MSVCRT:gs_report.obj
 0001:0000283c       ?__scrt_initialize_thread_safe_statics@@YAHXZ 000000018000383c f   MSVCRT:thread_safe_statics.obj
 0001:0000290c       ?__scrt_uninitialize_thread_safe_statics@@YAXXZ 000000018000390c f   MSVCRT:thread_safe_statics.obj
 0001:000029b0       $$000000                   00000001800039b0     MSVCRT:amdsecgs.obj
 0001:000029e0       ?dllmain_crt_dispatch@@YAHQEAUHINSTANCE__@@KQEAX@Z 00000001800039e0 f   MSVCRT:dll_dllmain.obj
 0001:00002a30       ?dllmain_crt_process_attach@@YAHQEAUHINSTANCE__@@QEAX@Z 0000000180003a30 f   MSVCRT:dll_dllmain.obj
 0001:00002b48       ?dllmain_crt_process_detach@@YAH_N@Z 0000000180003b48 f   MSVCRT:dll_dllmain.obj
 0001:00002bcc       ?dllmain_dispatch@@YAHQEAUHINSTANCE__@@KQEAX@Z 0000000180003bcc f   MSVCRT:dll_dllmain.obj
 0001:000035e0       $$000000                   00000001800045e0     MSVCRT:guard_dispatch.obj
 0001:00003600       $$000000                   0000000180004600     MSVCRT:guard_xfg_dispatch.obj
 0001:00003616       ?fin$0@?0??dllmain_crt_process_attach@@YAHQEAUHINSTANCE__@@QEAX@Z@4HA 0000000180004616 f   MSVCRT:dll_dllmain.obj
 0001:0000362d       ?fin$0@?0??dllmain_crt_process_detach@@YAH_N@Z@4HA 000000018000462d f   MSVCRT:dll_dllmain.obj
 0001:00003646       ?fin$1@?0??dllmain_crt_process_detach@@YAH_N@Z@4HA 0000000180004646 f   MSVCRT:dll_dllmain.obj
 0001:0000365a       ?filt$0@?0??dllmain_dispatch@@YAHQEAUHINSTANCE__@@KQEAX@Z@4HA 000000018000465a f   MSVCRT:dll_dllmain.obj
 0001:00003690       __scrt_is_nonwritable_in_current_image$filt$0 0000000180004690 f   MSVCRT:utility.obj
 0002:00000218       ?__scrt_initialize_tss_var@@3P6AHXZEA 0000000180005218     MSVCRT:thread_safe_statics.obj
 0002:00000350       ?opcLengths@@3QBEB         0000000180005350     liblocaltab005.obj
 0002:00002518       GS_ExceptionPointers       0000000180007518     MSVCRT:gs_report.obj
 0002:00002c18       $unwind$fprintf            0000000180007c18     liblocaltab005.obj
 0002:00002c24       $unwind$printf             0000000180007c24     liblocaltab005.obj
 0002:00002c30       $unwind$?NewObject@JNIEnv_@@QEAAPEAV_jobject@@PEAV_jclass@@PEAU_jmethodID@@ZZ 0000000180007c30     liblocaltab005.obj
 0002:00002c30       $unwind$nsk_lcomplain      0000000180007c30     liblocaltab005.obj
 0002:00002c30       $unwind$nsk_ldisplay       0000000180007c30     liblocaltab005.obj
 0002:00002c38       $unwind$nsk_lvdisplay      0000000180007c38     liblocaltab005.obj
 0002:00002c38       $unwind$_RTC_Initialize    0000000180007c38     MSVCRT:initsect.obj
 0002:00002c38       $unwind$_RTC_Terminate     0000000180007c38     MSVCRT:initsect.obj
 0002:00002c38       $unwind$?__scrt_initialize_thread_safe_statics@@YAHXZ 0000000180007c38     MSVCRT:thread_safe_statics.obj
 0002:00002c44       $unwind$nsk_complain       0000000180007c44     liblocaltab005.obj
 0002:00002c44       $unwind$nsk_printf         0000000180007c44     liblocaltab005.obj
 0002:00002c4c       $unwind$nsk_lvcomplain     0000000180007c4c     liblocaltab005.obj
 0002:00002c64       $unwind$nsk_ltrace         0000000180007c64     liblocaltab005.obj
 0002:00002c64       $unwind$__report_gsfailure 0000000180007c64     MSVCRT:gs_report.obj
 0002:00002c6c       $unwind$Java_nsk_jvmti_GetLocalVariableTable_localtab005_check 0000000180007c6c     liblocaltab005.obj
 0002:00002c6c       $unwind$nsk_lvtrace        0000000180007c6c     liblocaltab005.obj
 0002:00002c6c       $unwind$__raise_securityfailure 0000000180007c6c     MSVCRT:gs_report.obj
 0002:00002c6c       $unwind$__scrt_initialize_crt 0000000180007c6c     MSVCRT:utility.obj
 0002:00002c6c       $unwind$__scrt_initialize_onexit_tables 0000000180007c6c     MSVCRT:utility.obj
 0002:00002c6c       $unwind$__scrt_release_startup_lock 0000000180007c6c     MSVCRT:utility.obj
 0002:00002c6c       $unwind$__scrt_uninitialize_crt 0000000180007c6c     MSVCRT:utility.obj
 0002:00002c6c       $unwind$_onexit            0000000180007c6c     MSVCRT:utility.obj
 0002:00002c74       $unwind$nsk_lverify        0000000180007c74     liblocaltab005.obj
 0002:00002c84       $unwind$nsk_vprintf        0000000180007c84     liblocaltab005.obj
 0002:00002c94       $unwind$?nsk_jni_lverify@@YAHHPEAUJNIEnv_@@HQEBDH1ZZ 0000000180007c94     liblocaltab005.obj
 0002:00002ca8       $unwind$?nsk_jni_check_exception@@YAHPEAUJNIEnv_@@QEBDH@Z 0000000180007ca8     liblocaltab005.obj
 0002:00002cc4       $unwind$nsk_jvmti_parseOptions 0000000180007cc4     liblocaltab005.obj
 0002:00002ce0       $unwind$nsk_jvmti_createJVMTIEnv 0000000180007ce0     liblocaltab005.obj
 0002:00002cf4       $unwind$Java_nsk_jvmti_unit_FollowReferences_FollowRefObjects_resetTags 0000000180007cf4     liblocaltab005.obj
 0002:00002cf4       $unwind$addRefToVerify     0000000180007cf4     liblocaltab005.obj
 0002:00002cf4       $unwind$nsk_jvmti_resetAgentData 0000000180007cf4     liblocaltab005.obj
 0002:00002cf4       $unwind$nsk_jvmti_setFailStatus 0000000180007cf4     liblocaltab005.obj
 0002:00002cf4       $unwind$__scrt_initialize_default_local_stdio_options 0000000180007cf4     MSVCRT:default_local_stdio_options.obj
 0002:00002cf4       $unwind$?dllmain_crt_dispatch@@YAHQEAUHINSTANCE__@@KQEAX@Z 0000000180007cf4     MSVCRT:dll_dllmain.obj
 0002:00002cf4       $unwind$DllMain            0000000180007cf4     MSVCRT:dll_dllmain_stub.obj
 0002:00002cf4       $unwind$__GSHandlerCheck   0000000180007cf4     MSVCRT:gshandler.obj
 0002:00002cf4       $unwind$?__scrt_uninitialize_thread_safe_statics@@YAXXZ 0000000180007cf4     MSVCRT:thread_safe_statics.obj
 0002:00002cf4       $unwind$__scrt_acquire_startup_lock 0000000180007cf4     MSVCRT:utility.obj
 0002:00002cf4       $unwind$__scrt_dllmain_after_initialize_c 0000000180007cf4     MSVCRT:utility.obj
 0002:00002cf4       $unwind$__scrt_dllmain_before_initialize_c 0000000180007cf4     MSVCRT:utility.obj
 0002:00002cf4       $unwind$__scrt_dllmain_crt_thread_attach 0000000180007cf4     MSVCRT:utility.obj
 0002:00002cf4       $unwind$__scrt_dllmain_crt_thread_detach 0000000180007cf4     MSVCRT:utility.obj
 0002:00002cf4       $unwind$__scrt_dllmain_uninitialize_c 0000000180007cf4     MSVCRT:utility.obj
 0002:00002cf4       $unwind$__scrt_dllmain_uninitialize_critical 0000000180007cf4     MSVCRT:utility.obj
 0002:00002cf4       $unwind$atexit             0000000180007cf4     MSVCRT:utility.obj
 0002:00002cfc       $unwind$nsk_jvmti_lverify  0000000180007cfc     liblocaltab005.obj
 0002:00002d10       $unwind$exitOnError        0000000180007d10     liblocaltab005.obj
 0002:00002d20       $unwind$check_option       0000000180007d20     liblocaltab005.obj
 0002:00002d20       $unwind$_DllMainCRTStartup 0000000180007d20     MSVCRT:dll_dllmain.obj
 0002:00002d30       $unwind$Java_nsk_share_jvmti_ArgumentHandler_getAgentOptionsString 0000000180007d30     liblocaltab005.obj
 0002:00002d44       $unwind$Java_nsk_jvmti_unit_FollowReferences_FollowRefObjects_getTag 0000000180007d44     liblocaltab005.obj
 0002:00002d44       $unwind$Java_nsk_share_jvmti_DebugeeClass_checkStatus 0000000180007d44     liblocaltab005.obj
 0002:00002d44       $unwind$agentThreadWrapper 0000000180007d44     liblocaltab005.obj
 0002:00002d54       $unwind$Agent_Initialize   0000000180007d54     liblocaltab005.obj
 0002:00002d54       $unwind$startAgentThreadWrapper 0000000180007d54     liblocaltab005.obj
 0002:00002d70       $unwind$syncDebuggeeStatus 0000000180007d70     liblocaltab005.obj
 0002:00002d70       $unwind$__scrt_dllmain_exception_filter 0000000180007d70     MSVCRT:utility.obj
 0002:00002d84       $unwind$Java_nsk_share_jvmti_DebugeeClass_resetAgentData 0000000180007d84     liblocaltab005.obj
 0002:00002d8c       $unwind$MA_checkStatus     0000000180007d8c     liblocaltab005.obj
 0002:00002da0       $unwind$Java_nsk_jvmti_unit_FollowReferences_FollowRefObjects_setTag 0000000180007da0     liblocaltab005.obj
 0002:00002db8       $unwind$Java_nsk_jvmti_unit_FollowReferences_FollowRefObjects_addRefToVerify 0000000180007db8     liblocaltab005.obj
 0002:00002dd4       $unwind$checkAttr          0000000180007dd4     liblocaltab005.obj
 0002:00002dec       $unwind$capture_previous_context 0000000180007dec     MSVCRT:gs_report.obj
 0002:00002df8       $unwind$__GSHandlerCheckCommon 0000000180007df8     MSVCRT:gshandler.obj
 0002:00002e00       $xdatasym                  0000000180007e00     MSVCRT:amdsecgs.obj
 0002:00002e04       $unwind$?dllmain_crt_process_attach@@YAHQEAUHINSTANCE__@@QEAX@Z 0000000180007e04     MSVCRT:dll_dllmain.obj
 0002:00002e40       $unwind$?fin$0@?0??dllmain_crt_process_attach@@YAHQEAUHINSTANCE__@@QEAX@Z@4HA 0000000180007e40     MSVCRT:dll_dllmain.obj
 0002:00002e40       $unwind$?fin$0@?0??dllmain_crt_process_detach@@YAH_N@Z@4HA 0000000180007e40     MSVCRT:dll_dllmain.obj
 0002:00002e40       $unwind$?fin$1@?0??dllmain_crt_process_detach@@YAH_N@Z@4HA 0000000180007e40     MSVCRT:dll_dllmain.obj
 0002:00002e48       $unwind$?dllmain_crt_process_detach@@YAH_N@Z 0000000180007e48     MSVCRT:dll_dllmain.obj
 0002:00002e9c       $unwind$?dllmain_dispatch@@YAHQEAUHINSTANCE__@@KQEAX@Z 0000000180007e9c     MSVCRT:dll_dllmain.obj
 0002:00002ec4       $unwind$?filt$0@?0??dllmain_dispatch@@YAHQEAUHINSTANCE__@@KQEAX@Z@4HA 0000000180007ec4     MSVCRT:dll_dllmain.obj
 0002:00002ecc       $unwind$__scrt_is_nonwritable_in_current_image 0000000180007ecc     MSVCRT:utility.obj
 0002:00002eec       $unwind$__scrt_is_nonwritable_in_current_image$filt$0 0000000180007eec     MSVCRT:utility.obj
 0002:00002ef4       $unwind$__scrt_fastfail    0000000180007ef4     MSVCRT:utility_desktop.obj
 0002:00002f04       $unwind$__security_init_cookie 0000000180007f04     MSVCRT:gs_support.obj
 0002:00002f10       $unwind$__isa_available_init 0000000180007f10     MSVCRT:cpu_disp.obj
 0002:00002f20       $xdatasym                  0000000180007f20     MSVCRT:guard_dispatch.obj
 0002:00002f28       $xdatasym                  0000000180007f28     MSVCRT:guard_xfg_dispatch.obj
 0002:00002f30       .edata                     0000000180007f30     localtab005.exp
 0002:00002f58       rgpv                       0000000180007f58     localtab005.exp
 0002:00002f94       rgszName                   0000000180007f94     localtab005.exp
 0002:00002fd0       rgwOrd                     0000000180007fd0     localtab005.exp
 0002:00002fee       szName                     0000000180007fee     localtab005.exp
 0002:00002ffe       $N00001                    0000000180007ffe     localtab005.exp
 0002:0000300d       $N00002                    000000018000800d     localtab005.exp
 0002:0000301a       $N00003                    000000018000801a     localtab005.exp
 0002:00003051       $N00004                    0000000180008051     localtab005.exp
 0002:00003096       $N00005                    0000000180008096     localtab005.exp
 0002:000030d3       $N00006                    00000001800080d3     localtab005.exp
 0002:0000311b       $N00007                    000000018000811b     localtab005.exp
 0002:0000315b       $N00008                    000000018000815b     localtab005.exp
 0002:00003198       $N00009                    0000000180008198     localtab005.exp
 0002:000031d3       $N00010                    00000001800081d3     localtab005.exp
 0002:00003201       $N00011                    0000000180008201     localtab005.exp
 0002:00003232       $N00012                    0000000180008232     localtab005.exp
 0002:00003261       $N00013                    0000000180008261     localtab005.exp
 0002:00003290       $N00014                    0000000180008290     localtab005.exp
 0002:000032c5       $N00015                    00000001800082c5     localtab005.exp
 0002:0000372a       .idata$6                   000000018000872a     kernel32:KERNEL32.dll
 0002:0000378e       .idata$6                   000000018000878e     vcruntime:VCRUNTIME140.dll
 0002:00003920       .idata$6                   0000000180008920     ucrt:api-ms-win-crt-heap-l1-1-0.dll
 0002:00003940       .idata$6                   0000000180008940     ucrt:api-ms-win-crt-runtime-l1-1-0.dll
 0002:00003962       .idata$6                   0000000180008962     ucrt:api-ms-win-crt-convert-l1-1-0.dll
 0002:00003984       .idata$6                   0000000180008984     ucrt:api-ms-win-crt-stdio-l1-1-0.dll
 0002:000039a4       .idata$6                   00000001800089a4     ucrt:api-ms-win-crt-string-l1-1-0.dll
 0003:00000000       constr_lv                  0000000180009000     liblocaltab005.obj
 0003:000000b0       insMeth_lv                 00000001800090b0     liblocaltab005.obj
 0003:00000160       statMeth_lv                0000000180009160     liblocaltab005.obj
 0003:000001d8       ?codeAttributeName@@3PEBDEB 00000001800091d8     liblocaltab005.obj
 0003:000001e0       ?lineNumberAttributeName@@3PEBDEB 00000001800091e0     liblocaltab005.obj
 0003:000001e8       ?localVarAttributeName@@3PEBDEB 00000001800091e8     liblocaltab005.obj
 0003:000001f0       ?localVarTypeAttributeName@@3PEBDEB 00000001800091f0     liblocaltab005.obj
 0003:000001f8       ?stackMapAttributeName@@3PEBDEB 00000001800091f8     liblocaltab005.obj
 0003:00000200       ?callBytes@@3PAEA          0000000180009200     liblocaltab005.obj
 0003:00000204       ?allocBytes@@3PAEA         0000000180009204     liblocaltab005.obj
 0003:00000210       methInfo                   0000000180009210     liblocaltab005.obj
 0003:0001ad44       redefineAttempted          0000000180023d44     liblocaltab005.obj
 0003:0001ad48       nsk_context                0000000180023d48     liblocaltab005.obj
 0003:0001ad54       redefineSucceed            0000000180023d54     liblocaltab005.obj
 0003:0001ad58       agentFailed                0000000180023d58     liblocaltab005.obj
 0003:0001ad5c       currentAgentStatus         0000000180023d5c     liblocaltab005.obj
 0003:0001ad60       context                    0000000180023d60     liblocaltab005.obj
 0003:0001ae18       agentThread                0000000180023e18     liblocaltab005.obj
 0003:0001ae20       agentThreadProc            0000000180023e20     liblocaltab005.obj
 0003:0001ae28       agentThreadArg             0000000180023e28     liblocaltab005.obj
 0003:0001ae30       agent_data                 0000000180023e30     liblocaltab005.obj
 0003:0001ae40       jvmti_env                  0000000180023e40     liblocaltab005.obj
 0003:0001ae48       jvm                        0000000180023e48     liblocaltab005.obj
 0003:0001ae50       jni_env                    0000000180023e50     liblocaltab005.obj
 0003:0001ae58       checkStatus_func           0000000180023e58     liblocaltab005.obj
 0003:0001ae60       ?codeAttributeIndex@@3GA   0000000180023e60     liblocaltab005.obj
 0003:0001ae64       ?lineNumberAttributeIndex@@3GA 0000000180023e64     liblocaltab005.obj
 0003:0001ae68       ?localVarAttributeIndex@@3GA 0000000180023e68     liblocaltab005.obj
 0003:0001ae6c       ?localVarTypeAttributeIndex@@3GA 0000000180023e6c     liblocaltab005.obj
 0003:0001ae70       ?stackMapAttributeIndex@@3GA 0000000180023e70     liblocaltab005.obj
 0003:0001ae74       ?stackFrameOffset@@3GA     0000000180023e74     liblocaltab005.obj
 0003:0001ae78       ?mode@@3HA                 0000000180023e78     liblocaltab005.obj
 0003:0001ae7c       ?constantPoolSize@@3GA     0000000180023e7c     liblocaltab005.obj
 0003:0001ae80       ?orig@@3PEBEEB             0000000180023e80     liblocaltab005.obj
 0003:0001ae88       ?gen@@3PEAEEA              0000000180023e88     liblocaltab005.obj
 0003:0001ae90       ?inputPos@@3PEAEEA         0000000180023e90     liblocaltab005.obj
 0003:0001ae98       ?endPos@@3PEBEEB           0000000180023e98     liblocaltab005.obj
 0003:0001aea0       ?genPos@@3PEAEEA           0000000180023ea0     liblocaltab005.obj
 0003:0001aea8       ?markPos@@3PEAEEA          0000000180023ea8     liblocaltab005.obj
 0003:0001aeb0       ?constantPool@@3PEAPEADEA  0000000180023eb0     liblocaltab005.obj
 0003:0001aeb8       ?constantPoolCount@@3GA    0000000180023eb8     liblocaltab005.obj
 0003:0001aebc       ?zeroBytes@@3PAEA          0000000180023ebc     liblocaltab005.obj
 0003:0001aec0       ?codeLength@@3IA           0000000180023ec0     liblocaltab005.obj
 0003:0001aec8       ?map@@3PEAIEA              0000000180023ec8     liblocaltab005.obj
 0003:0001aed0       ?widening@@3PEACEA         0000000180023ed0     liblocaltab005.obj
 0003:0001aed8       jvmti                      0000000180023ed8     liblocaltab005.obj
 0003:0001aee0       caps                       0000000180023ee0     liblocaltab005.obj
 0003:0001af00       GS_ExceptionRecord         0000000180023f00     MSVCRT:gs_report.obj
 0003:0001afa0       GS_ContextRecord           0000000180023fa0     MSVCRT:gs_report.obj
 0003:0001b470       ?g_tss_cv@@3U_RTL_CONDITION_VARIABLE@@A 0000000180024470     MSVCRT:thread_safe_statics.obj
 0003:0001b478       ?g_tss_event@@3PEAXEA      0000000180024478     MSVCRT:thread_safe_statics.obj
 0003:0001b480       ?g_tss_mutex@@3U_RTL_CRITICAL_SECTION@@A 0000000180024480     MSVCRT:thread_safe_statics.obj
 0003:0001b4a8       ?g_sleep_condition_variable_cs@@3P6AHPEAU_RTL_CONDITION_VARIABLE@@PEAU_RTL_CRITICAL_SECTION@@K@ZEA 00000001800244a8     MSVCRT:thread_safe_statics.obj
 0003:0001b4b0       ?g_wake_all_condition_variable@@3P6AXPEAU_RTL_CONDITION_VARIABLE@@@ZEA 00000001800244b0     MSVCRT:thread_safe_statics.obj
 0003:0001b4bc       ?__proc_attached@@3HA      00000001800244bc     MSVCRT:dll_dllmain.obj
 0003:0001b4d0       ?is_initialized_as_dll@@3_NA 00000001800244d0     MSVCRT:utility.obj
 0003:0001b4d1       ?module_local_atexit_table_initialized@@3_NA 00000001800244d1     MSVCRT:utility.obj
 0003:0001b4d8       ?module_local_atexit_table@@3U_onexit_table_t@@A 00000001800244d8     MSVCRT:utility.obj
 0003:0001b4f0       ?module_local_at_quick_exit_table@@3U_onexit_table_t@@A 00000001800244f0     MSVCRT:utility.obj
